:03F0000002F00813
:03F0610002F003B7
:05F0030012F06480FE24
:02F064007A0030
:03F06600BA4000AD
:0DF06900500B8A827583FE74FFF00A80F060
:07F076007A00C2A875E10455
:0BF07D0090DF3BE0FBBB01F875E102F7
:0EF0880090DF3BE0FBBB0DF88A030A7CFE9094
:09F09600DF02E0FD8B828C83F0A7
:0AF09F0090DF02E0FBC3EA9B501370
:05F0A90010890280FB4C
:0EF0AE008A030A8B827583FEE5D9FBF080E3AE
:0EF0BC0075E10490FE01E0FABADD9D90FE02BF
:07F0CA00E0FABA5595A522FA
:06F03700E478FFF6D8FDAD
:08F015007900E94400601B7A58
:05F01D000090F0D57821
:03F02200007593E3
:0AF0250000E493F2A308B80002050E
:08F02F0093D9F4DAF27593FFA6
:08F03D007800E84400600A7944
:03F04500007593C0
:06F0480000E4F309D8FC0E
:08F04E007800E84400600C7931
:0BF0560000900000E4F0A3D8FCD9FA01
:03F0080075810708
:0AF00B0012F0D1E582600302F00369
:04F0D1007582002222
:00000001FF
